:100000000C94D7010C94F4010C94F4010C94F401B9
:100010000C94F4010C94F4010C94F4010C94F4018C
:100020000C94F4010C94D30C0C94F4010C94E00D9A
:100030000C94F4010C94F4010C94F4010C94F4016C
:100040000C94F4010C94F4010C94180C0C94DC0B3B
:100050000C94F4010C94F4010C94F4010C94F4014C
:100060000C94F4010C94F401084AD73B3BCE016E8A
:1000700084BCBFFDC12F3D6C74319ABD56833DDAFF
:100080003D00C77F11BED9E4BB4C3E916BAAAABE0E
:10009000000000803F05A84CCDB2D44EB93836A937
:1000A000020C50B9918688083CA6AAAA2ABE000074
:1000B00000803F0D0A00466C6F6174696E672070A6
:1000C0006F696E74206572726F720D0A00556E73DF
:1000D0007570706F727465642073746174656D659A
:1000E0006E740D0A00457870656374656420636FF3
:1000F0006D6D616E64206C65747465720D0A0042EA
:100100006164206E756D62657220666F726D6174D8
:100110000D0A006572726F723A20006F6B0D0A0053
:100120000D0A000D0A4772626C20302E37640057AA
:1001300061726E696E673A204661696C656420740D
:100140006F207265616420454550524F4D207365A4
:100150007474696E67732E205573696E67206465C9
:100160006661756C74732E0D0A0027242720746F46
:100170002064756D702063757272656E742073658E
:100180007474696E67730D0A0053746F726564202E
:100190006E65772073657474696E670D0A00556E1D
:1001A0006B6E6F776E20706172616D657465720D34
:1001B0000A00537465702070756C7365206D7573DB
:1001C00074206265203E3D2033206D6963726F7339
:1001D00065636F6E64730D0A0053746570732F6DE1
:1001E0006D206D757374206265203E20302E300DB9
:1001F0000A000D0A2724783D76616C756527207406
:100200006F2073657420706172616D657465722012
:100210006F72206A7573742027242720746F2064FE
:10022000756D702063757272656E74207365747479
:10023000696E67730D0A002028636F726E657269BC
:100240006E67206A756E6374696F6E206465766987
:100250006174696F6E20696E206D6D2900202861C0
:100260006363656C65726174696F6E20696E206D81
:100270006D2F7365635E32290D0A2439203D2000FD
:10028000290D0A2438203D20002028737465702031
:10029000706F727420696E76657274206D61736B15
:1002A0002E2062696E617279203D200020286D6DDC
:1002B0002F617263207365676D656E74290D0A2462
:1002C00037203D200020286D6D2F6D696E206465FC
:1002D0006661756C74207365656B20726174652945
:1002E0000D0A2436203D200020286D6D2F6D696E8B
:1002F0002064656661756C74206665656420726152
:100300007465290D0A2435203D200020286D69637D
:10031000726F7365636F6E647320737465702070A1
:10032000756C7365290D0A2434203D200020287344
:10033000746570732F6D6D207A290D0A2433203D6A
:100340002000202873746570732F6D6D2079290D3E
:100350000A2432203D2000202873746570732F6DAD
:100360006D2078290D0A2431203D20002430203DC5
:100370002000494E46494E4954594E414ECDCCCCB1
:100380003D0AD7233C17B7D13877CC2B329595E669
:10039000241FB14F0A000020410000C84200401C49
:1003A0004620BCBE4CCA1B0E5AAEC59D740011241B
:1003B0001FBECFEFD8E0DEBFCDBF11E0A0E0B1E0BF
:1003C000E0E0F6E402C005900D92A030B107D9F745
:1003D00016E0A0E0B1E001C01D92A93FB107E1F72E
:1003E0000E946E030C94FE220C940000A0E0B0E08A
:1003F000ECEFF1E00C94CD22EC015B01611571058D
:1004000019F0FB0191838083F9908F2D90E00E9479
:10041000BC22892BC9F7FDE2FF1621F4F990EE24E6
:10042000E39405C02BE2F21609F4F990EE248E0154
:1004300001501040C80162E773E043E050E00E94C1
:100440005603892B01F58E010E5F1F4FC80165E72A
:1004500073E045E050E00E945603892B19F48E01A9
:10046000095F1F4FA114B10419F0F5011183008336
:10047000E0FC04C070E090E080E814C070E090E020
:1004800080E86FEF08C1C8016AE773E043E050E01D
:100490000E945603892B69F4A114B10429F470E079
:1004A00090E080EC6FE7F7C02296F501D183C0831E
:1004B000F6CF8824992440E050E060E070E0EF2D12
:1004C000E053EA30A0F5F2E0EF2A8E2D90E09C0197
:1004D00028703070E2FE06C0232B79F50894811C49
:1004E000911C2BC0232B19F0089481089108DB0183
:1004F000CA0112E0880F991FAA1FBB1F1A95D1F7D6
:10050000480F591F6A1F7B1F440F551F661F771F17
:100510004E0F511D611D711D483929E9520729E906
:10052000620729E1720748F084E0E82A06C0EE3F3E
:1005300031F4E3FC39C098E0E92AF990C0CFE53303
:1005400011F0E53189F529912D3219F4E0E1EE2A17
:1005500005C02B3219F081E090E003C0299182E0C0
:1005600090E0E22FE053EA3018F0C81BD90B1CC012
:1005700020E030E0FCE020383F075CF4C901880F40
:10058000991F880F991F280F391F220F331F2E0F15
:10059000311DE991E053EA3068F3E4FE03C0309581
:1005A00021953F4F820E931ECE2CDD24E1FE07C025
:1005B000A114B10421F02197F501D183C083CB01AF
:1005C000BA010E94231F7B018C01F3E0CF22DD24BE
:1005D00023E0C216D10421F417FB109517F91095EA
:1005E00057016801C801B70120E030E040E050E069
:1005F0000E94831E882309F44AC097FE0DC021E99A
:10060000E22E23E0F22E9094819491089394C0E21C
:10061000D0E000E010E012C099EAE92E93E0F92E54
:10062000F6CFF7012591359145915491C601B50159
:100630000E9463215B016C018C1A9D0A8C169D0639
:1006400084F7D595C7950F5F1F4F0630110529F028
:100650008CEF9FEFE80EF91EF1CFC501D6017C01AA
:100660008D018C2D880F8D2D881F8F3F51F0C60175
:10067000B50120E030E040E050E00E94831E882376
:1006800031F482E290E09093F8068093F7067E2D95
:100690009F2D802F612F272F392F482F562FB901DB
:1006A000CA01CDB7DEB7ECE00C94E922FB01DC0116
:1006B0004150504088F08D9181341CF08B350CF402
:1006C000805E659161341CF06B350CF4605E861BB6
:1006D000611171F3990B0895881BFCCF789460E841
:1006E00075E280E090E00E94930B0E943C0C0E9417
:1006F0001C130E947F140E94550D0E94880B0E94BB
:10070000E8060E94D41B0E948C0CFDCF0E94BE0DF7
:1007100008952F923F924F925F926F927F928F92A5
:100720009F92AF92BF92CF92DF92EF92FF920F9380
:100730001F93DF93CF93CDB7DEB7CE54D0400FB623
:10074000F894DEBF0FBECDBF3C017EAF6DAF2196EA
:100750005FAF4EAF219722962FAF229723960FAF10
:1007600023972496EFAE24972896ACAEBDAECEAEBE
:10077000DFAE289729968FAE2997E22EFF24EE0C44
:10078000FF1CEE0CFF1C4E0D5F1D5CAF4BAFDA0182
:100790002D903D904D905C90FC01EE0DFF1DC2012F
:1007A000B10120813181428153810E94AA1D69AB30
:1007B0007AAB8BAB9CAB10E0000F111F000F111F29
:1007C0002196EEADFFAD2197E00FF11FFAAFE9AF33
:1007D000A080B180C280D380F301E00FF11FC60179
:1007E000B50120813181428153810E94AA1D6DA7EC
:1007F0007EA78FA798AB24962FAD2497E22FF0E029
:10080000EE0FFF1FEE0FFF1F6E0E7F1ED3018D91A7
:100810009D910D90BC91A02D8DAB9EABAFABB8AFB1
:100820002DAD3EADE20FF31F608171818281938116
:100830002DA93EA94FA958AD0E94A91D69A77AA765
:100840008BA79CA7D201C101B0588DA39EA3AFA3D3
:10085000B8A7A6019501505829A33AA34BA35CA3BE
:100860004DAD5EADE40EF51ED7016D917D918D917C
:100870009C9129A93AA94BA95CA90E94A91D3B01F9
:100880004C01EDADFEAD0E0F1F1FD8016D917D9196
:100890008D919C912DA53EA54FA558A90E94A91DFB
:1008A0005B016C016DA17EA18FA198A5A6019501A8
:1008B0000E9463217B018C0169A17AA18BA19CA17B
:1008C000A40193010E9463219B01AC01C801B701FF
:1008D0000E94A91D1B012C016DA17EA18FA198A5CD
:1008E000A40193010E9463217B018C0169A17AA17B
:1008F0008BA19CA1A60195010E9463219B01AC01E3
:10090000C801B7010E94AA1D9B01AC01C201B1013F
:100910000E941D1E5B016C0120E030E040E050E0D1
:100920000E94831E882354F4C601B5012BED3FE0DD
:1009300049EC50E40E94AA1D5B016C01A8968FADA2
:10094000A897882351F0C601B5012BED3FE049EC93
:1009500050E40E94A91D5B016C01C601B501A79678
:100960002CAD3DAD4EAD5FADA7970E94632129A58B
:100970003AA54BA55CA50E949E207B018C0120E03E
:1009800030E040E050E00E94831E882309F4CAC191
:10099000C801B7012091EB063091EC064091ED06BD
:1009A0005091EE060E948A1E0E94601F0E94F71E50
:1009B00078A36F8F2996BFAD2997BB23A1F080E064
:1009C00090E00E94231F9B01AC0128966CAD7DAD89
:1009D0008EAD9FAD28970E94632128966CAF7DAFA6
:1009E0008EAF9FAF28972F8D38A1B90180E090E09E
:1009F0000E94231F7B018C01C601B501A80197014C
:100A00000E948A1E6B8F7C8F8D8F9E8F69A57AA521
:100A10008BA59CA5A80197010E948A1E6F8B788FD9
:100A2000898F9A8F6B8D7C8D8D8D9E8D20E030E02F
:100A300040E05FEB0E9463212B8D3C8D4D8D5E8DE0
:100A40000E94632120E030E040E85FE30E94AA1D9D
:100A50006B8B7C8B8D8B9E8B24963FAD2497E32FE5
:100A6000F0E0EE0FFF1FEE0FFF1FCE010196E80F23
:100A7000F91F2DA93EA94FA958AD20833183428388
:100A8000538341E050E05E874D8766242296BFADD8
:100A90002297AB2FB0E0AA0FBB1FAA0FBB1FA80F56
:100AA000B91F2B96BFAFAEAF2B9723963FAD2397C1
:100AB000232F30E0220F331F220F331F280F391F3F
:100AC0002D963FAF2EAF2D972F96FFAFEEAF2F97FE
:100AD00003C148E146150CF446C06DA17EA18FA16B
:100AE00098A52B8D3C8D4D8D5E8D0E9463217B01E1
:100AF0008C0169A17AA18BA19CA12B893C894D898C
:100B00005E890E9463219B01AC01C801B7010E946C
:100B1000AA1D7B018C016DA17EA18FA198A52B89B7
:100B20003C894D895E890E9463215B016C0169A14A
:100B30007AA18BA19CA12B8D3C8D4D8D5E8D0E9449
:100B400063219B01AC01C601B5010E94A91D6DA3E3
:100B50007EA38FA398A76394C701D80189A39AA302
:100B6000ABA3BCA361C0AD85BE85BD0180E090E0B4
:100B70000E94231F2B8D3C8D4D8D5E8D0E94632125
:100B80007B018C01C8010E94871E6F87788B898B3F
:100B90009A8BB701C8010E94E6213B014C01EBADE5
:100BA000FCADE080F1800281138117FB109517F9ED
:100BB0001095A9ADBAAD2D903D904D905C90C801B7
:100BC000B7012F85388949895A890E9463215B01C1
:100BD0006C01C201B101A40193010E9463219B0138
:100BE000AC01C601B5010E94AA1D6DA37EA38FA30F
:100BF00098A7C801B701A40193010E9463217B015A
:100C00008C01C201B1012F85388949895A890E9416
:100C100063219B01AC01C801B7010E94A91D69A312
:100C20007AA38BA39CA3662469A97AA98BA99CA902
:100C30002DA13EA14FA158A50E94AA1D2B96EEAD55
:100C4000FFAD2B9760837183828393836DA57EA50F
:100C50008FA598A929A13AA14BA15CA10E94AA1D28
:100C60002D96AEADBFAD2D976D937D938D939C93D7
:100C700013972F96EEADFFAD2F9760817181828122
:100C800093812F89388D498D5A8D0E94AA1D2F96E8
:100C9000AEADBFAD2F976D937D938D939C931397BE
:100CA00069817A818B819C812D813E814F8158851C
:100CB000E984FA840B851C852896ACACBDACCEAC1F
:100CC000DFAC289729968FAC29970E947F16ED8577
:100CD000FE853196FE87ED872D853E854F8D58A187
:100CE0002417350708F4F5CEADADBEAD6D917D91FD
:100CF0008D919C91139714962D913D914D915C91FE
:100D000017971896ED90FD900D911C911B972896C2
:100D1000ACACBDACCEACDFAC289729968FAC299794
:100D20000E947F16C25BDF4F0FB6F894DEBF0FBE86
:100D3000CDBFCF91DF911F910F91FF90EF90DF908A
:100D4000CF90BF90AF909F908F907F906F905F906B
:100D50004F903F902F900895EF92FF920F931F9323
:100D6000CF93DF937B018C010E94601F0E94F71ECE
:100D7000EB010E94D30DBE0180E090E00E94231F92
:100D80009B01AC01C801B7010E94A91D20E030E021
:100D90004AE754E40E9463210E94601F0E94F71EEC
:100DA000DC01CB010E94861B20E931E008C080E114
:100DB00097E2F9013197F1F70197D9F72197209739
:100DC000B1F7DF91CF911F910F91FF90EF900895B0
:100DD00081E2E0E0F1E0DF011D928A95E9F7809180
:100DE000E2069091E306A091E406B091E5068093B7
:100DF000070190930801A0930901B0930A01809123
:100E0000E6069091E706A091E806B091E906809386
:100E10000B0190930C01A0930D01B0930E01109261
:100E20001E0191E090931F0182E080932001909336
:100E3000040108952F923F924F925F926F927F929A
:100E40008F929F92AF92BF92CF92DF92EF92FF92DA
:100E50000F931F93DF93CF93CDB7DEB7AA970FB64B
:100E6000F894DEBF0FBECDBF2C0119821092000195
:100E70001BA21AA262E0662E712C6C0E7D1E4E0122
:100E80000894811C911C53E0A52ECC24C39442E00D
:100E9000B42E34E0332E22242A94DAC025313105D1
:100EA00009F489C02631310584F52430310509F46F
:100EB0005BC025303105A4F42130310509F45AC056
:100EC0002230310524F4232B09F451C0B4C0223060
:100ED000310509F452C02330310509F0ACC050C0CF
:100EE0002231310509F456C0233131052CF421316A
:100EF000310509F0A0C047C02331310509F451C0C4
:100F00002431310509F097C053C02A35310509F461
:100F10005BC02B353105A4F42E31310511F12F3191
:100F200031052CF42C31310509F085C01AC0253368
:100F3000310509F443C02035310509F07CC041C0BA
:100F40002C35310509F446C02C3531050CF43FC071
:100F50002D35310509F441C02E35310509F06BC03E
:100F60003FC042E04AA370C051E05AA36DC0109246
:100F700001016AC0C092010167C0B092010164C062
:100F8000A092010161C010921E01C0921F01B09297
:100F900020015AC010921E01B0921F01C092200180
:100FA00053C0C0921E01B0921F01109220014CC08C
:100FB000C092030149C01092030146C061E06BA3D7
:100FC00043C03092010140C0C09204013DC0109264
:100FD00004013AC073E07AA337C0C092020134C062
:100FE0001092020131C023303105E1F02430310587
:100FF00034F477FD20C02230310574F010C0253064
:101000003105B1F02530310584F02E31310539F04C
:101010002C33310581F403C0C092050115C0B09294
:10102000050112C0C09206010FC0209206010CC03B
:101030001092060109C0A092000106C0C801B701C4
:101040000E94F71E60931B01809100018823D1F458
:101050009981F201E90FF11DD080DD2099F08D2DED
:1010600081548A3110F082E00BC09F5F9983C201E6
:10107000B401A3010E94991B892B09F007C381E0E9
:101080008093000180910001882309F0E6C2198253
:10109000FE0136968CE0DF01482F1D924A95E9F754
:1010A0009E012E5E3F4FD9011D928A95E9F7AFE070
:1010B000B1E08CE00D9001928150E1F71FA218A6DB
:1010C000B0E8B9A7EFEBEAA71CA21DA21EA222243A
:1010D000332440E050E060E070E04E8F5F8F68A303
:1010E00079A33E010894611C711CACC0C701B60114
:1010F00023E333E34BEC51E40E9463214B015C0199
:101100000035E1F001355CF40634E1F006340CF40E
:1011100099C0802F8954833008F094C03FC00335B4
:1011200009F454C0043524F4023509F08BC047C0DB
:10113000802F8855833008F085C051C0CDA2DEA233
:10114000170180C0C501B40120E030E040E050E06C
:101150000E94831E18161CF051E0509300018091EC
:101160000201882329F08FA298A6A9A6BAA66AC070
:1011700080910101882349F480920B0190920C0127
:10118000A0920D01B0920E015DC080920701909275
:101190000801A0920901B0920A0154C0E02FFF2774
:1011A000E7FDF095E954F040EE0FFF1FEE0FFF1F33
:1011B000E60DF71D818A928AA38AB48A43C08E8E77
:1011C0009F8EA8A2B9A261E06CA33CC0C701B60182
:1011D0000E94F21E70931D0160931C0133C0809128
:1011E0000401882319F47BA1772389F0E02FFF27DE
:1011F000E7FDF095E855F040EE0FFF1FEE0FFF1FE3
:10120000E60DF71D85829682A782B0861BC0112746
:1012100007FD109508551040000F111F000F111FFA
:10122000060D171DD80115966D917D918D919C919C
:101230001897A50194010E94AA1DF8016583768381
:10124000878390879981F201E90FF11D00810023C6
:10125000A9F0802F81548A3110F082E00DC09F5F89
:101260009983C201B301AE014E5F5F4F0E94991B8B
:10127000892B09F023C281E0809300018091000155
:10128000882309F0EAC18091060140911C01509128
:101290001D01662757FD6095762F992787FD90954C
:1012A0000E946A0BFAA1F13091F0F13030F1F23086
:1012B00021F0F33009F0C6C111C00E9486038CE012
:1012C000FE013696DF011D928A95E9F7BBC12DA17B
:1012D0003EA1B901C1010E94AC06B4C16E817F81FB
:1012E000888599852A853B854C855D85EE84FF84BC
:1012F000088919890E940B14A5C1B0900101B1E0C1
:10130000BB16E9F0BB1628F0E3E0EB1508F49AC130
:101310003BC06E817F81888599852A853B854C8578
:101320005D85EE84FF8408891989A0900B01B09037
:101330000C01C0900D01D0900E01882422C06E8156
:101340007F81888599852A853B854C855D85EE84DE
:10135000FF840889198980900201882061F4F09146
:101360000701FFA3A0910801A8A7B0910901B9A79F
:10137000E0910A01EAA7EFA1F8A5A9A5BAA55F0126
:101380006D010E947F165EC18E010F5F1F4FFCA191
:10139000FF2309F4EEC0E0911E01F0E0EE0FFF1F05
:1013A000EE0FFF1FD801AE0FBF1FE050FF4F159685
:1013B0006D917D918D919C911897278530894189F8
:1013C00052890E94A91D1B012C01E0911F01F0E030
:1013D000EE0FFF1FEE0FFF1F0E0F1F1FE050FF4FFE
:1013E000D80115966D917D918D919C9118972785C7
:1013F0003089418952890E94A91D3B014C018CE032
:10140000FE017296DF011D928A95E9F76E8D7F8D40
:1014100088A199A120E030E040E850E40E946321D7
:101420002E8D3F8D48A159A10E9463217B018C0123
:10143000C201B101A20191010E9463219B01AC0193
:10144000C801B7010E94A91D7B018C01C401B30131
:10145000A40193010E9463219B01AC01C801B70163
:101460000E94A91D0E94F0217B018C01C201B101E3
:10147000A40193010E949E209B01AC0117FB1095D3
:1014800017F91095C801B7010E948A1E6B017C01F3
:10149000A70196010E944422882321F084E08093D2
:1014A0000001DBC0B3E0BB1621F4F7FAF094F7F8C3
:1014B000F0946E8D7F8D88A199A120E030E040E00E
:1014C00050E00E94831E88236CF4F7FAF094F7F83A
:1014D000F0944E8D5F8D68A179A170584E8F5F8F0B
:1014E00068A379A300911E01A02EBB24AA0CBB1CEB
:1014F000AA0CBB1C8E010F5F1F4FA00EB11EC401B2
:10150000B301A70196010E9463219B01AC01C201B6
:10151000B1010E94A91D20E030E040E05FE30E949D
:101520006321D50151966D937D938D939C93549730
:1015300080911F0190E0880F991F880F991F080F55
:10154000191FC201B101A70196010E9463219B01ED
:10155000AC01C401B3010E94AA1D20E030E040E0CC
:101560005FE30E946321F801618B728B838B948B04
:1015700023C0E0911E01F0E0EE0FFF1FEE0FFF1FF2
:10158000E00FF11F618972898389948920911F017D
:1015900030E0220F331F220F331F020F131FD80119
:1015A00051962D913D914D915C9154970E949E20B2
:1015B0006E8F7F8F88A399A39091010120911E01C6
:1015C00000911F01E090200180900201882061F4C9
:1015D000B0910701BFA3E0910801E8A7F0910901CC
:1015E000F9A740910A014AA700D000D00F92EDB7A9
:1015F000FEB731964E8D5F8D68A179A1ADB7BEB7AC
:1016000011964D935D936D937C93149780E0923087
:1016100009F481E084838FE091E0BE016A5F7F4F2F
:10162000AE014E5E5F4F3FA1E8A5F9A5AAA5A32E86
:10163000BE2ECF2EDA2E0E9489030F900F900F90AE
:101640000F900F90AFE0B1E0FE0136968CE0019074
:101650000D928150E1F780910001AA960FB6F8949F
:10166000DEBF0FBECDBFCF91DF911F910F91FF90D5
:10167000EF90DF90CF90BF90AF909F908F907F9032
:101680006F905F904F903F902F9008956A817B817B
:101690008C819D810E943D227B018C010E94F21E63
:1016A0009B01BDE4DB1609F49ECCE4E5DE1609F4EB
:1016B000C5CCF7E4DF1609F0C7CCF0CBCA80DB80DD
:1016C000EC80FD8080910301882309F00FCD460155
:1016D000570116CDCF93DF93EC01809121019091BA
:1016E0002201C817D90789F00E94D30D209741F035
:1016F0001C161D0614F42D9801C02D9A2C9A01C0B9
:101700002C98D0932201C0932101DF91CF910895AD
:10171000249A259A80E090E040E050E060E070E09C
:101720000E946A0B0895EF92FF920F931F937B0123
:101730008C0122E030E040E050E00E94A122205CD9
:101740003D4B404F5F4FCA01B901A80197010E946C
:10175000A122215030403093C5002093C400E0EC1A
:10176000F0E080818D7F8083E1ECF0E0808180611A
:1017700080838081886080838081806880831F91DE
:101780000F91FF90EF900895282FE09125019E2F53
:101790009F5F903109F490E0809126019817E1F362
:1017A000F0E0EC53F94F2083909325018091C10024
:1017B00080628093C10008951F920F920FB60F921E
:1017C00011248F939F93EF93FF9380912601E82F2D
:1017D000F0E0EC53F94F90819093C600982F9F5FF3
:1017E000903109F490E080912501981729F48091B7
:1017F000C1008F7D8093C10090932601FF91EF91EE
:101800009F918F910F900FBE0F901F901895909100
:10181000240180912301891711F48FEF0895E92F96
:10182000F0E0EC53FA4F80819F5F9093240108957C
:101830001F920F920FB60F9211242F938F939F93A5
:10184000EF93FF932091C600E09123019E2F9F5FAD
:1018500080912401981731F0F0E0EC53FA4F208387
:1018600090932301FF91EF919F918F912F910F9072
:101870000FBE0F901F9018951092590110925A01A7
:1018800083E291E00E949B1D80E291E00E949B1DFB
:101890000895CF93DF93EC01009719F48BE191E069
:1018A0002AC083E191E00E949B1DC230D10589F0DE
:1018B000C330D10524F4C130D105A1F407C0C33031
:1018C000D10551F0C430D10569F409C08FEF90E023
:1018D00012C085EE90E00FC08DEC90E00CC086EB5E
:1018E00090E009C0BE01882777FD8095982F0E945F
:1018F0007B1D83EB90E00E949B1DDF91CF910895AB
:10190000FC018081843221F4CF010E948813089564
:10191000CF010E941A0708951F9311E03DC02D309A
:10192000A9F4E0915901EE2351F0F0E0E95DFE4F9A
:10193000108287E291E00E94800C90E002C080E07B
:1019400090E00E94490C1092590106C080915A0102
:10195000882329F0293201F510925A011DC0213245
:10196000DCF02F32C9F0283219F410935A0114C058
:1019700090915901913380F4822F8156E92FF0E044
:101980009F5F8A3120F4E95DFE4F205202C0E95D7D
:10199000FE4F2083909359010E94070C282F8A3014
:1019A00009F4BFCFBCCF1F920F920FB60F92112434
:1019B0008F939F939BB18091EA068C71937E892BC4
:1019C0008BB91092B1009F918F910F900FBE0F9025
:1019D0001F9018959B01AC01203283E0380780E00E
:1019E000480780E0580720F420E233E040E050E070
:1019F00060E070E788E399E30E947F22C901DA0181
:101A0000803020E0920721E0A20720E0B20738F4FE
:101A1000FC019C0140E050E060E070E031C08030AB
:101A200020E0920728E0A20720E0B207A8F473E0C4
:101A3000B695A795979587957A95D1F7FC019C0166
:101A400040E050E063E0220F331F441F551F6A95AA
:101A5000D1F761E070E014C026E0B695A7959795A0
:101A600087952A95D1F7FC019C0140E050E086E083
:101A7000220F331F441F551F8A95D1F762E070E093
:101A800080918100962F9F5F887F982B9093810093
:101A9000F0938900E093880020936F0130937001E8
:101AA000409371015093720108958AB18C6F8AB985
:101AB0008BB183709091EA06892B8BB9209A809123
:101AC00081008F7E80938100809181008860809367
:101AD0008100809180008D7F8093800080918000C4
:101AE0008E7F80938000809180008F738093800030
:101AF000809180008F7C809380001092B0001092C3
:101B0000B1008091700081608093700060E273E0AA
:101B100080E090E00E94EA0C109273011092740130
:101B2000109275011092760110925C0110925B0187
:101B300010926E0110927F0180916F008D7F8093D3
:101B40006F008AEF90E020E931E0F9013197F1F779
:101B50000197D9F7289A089580917F01882369F425
:101B600081E080937F018091EA0680935D0128984F
:101B700080916F00826080936F000895EF92FF92D2
:101B80000F931F930E94421C60E070E080E090E0A1
:101B90009B01AC017B018C010E940B141F910F91E2
:101BA000FF90EF90089507C083B7816083BF889549
:101BB00083B78E7F83BF0E94F813892BA9F70895FE
:101BC0001F920F920FB60F921124EF92FF920F9374
:101BD0001F932F933F934F935F936F937F938F93B5
:101BE0009F93AF93BF93CF93DF93EF93FF93809136
:101BF0006E01882309F084C29BB120915D01822F80
:101C0000807E9F71892B8BB98BB1837E822B8BB9A0
:101C10008091E10690E0A0E0B0E00297A109B1094F
:101C2000880F991FAA1FBB1F81958093B20082E085
:101C30008093B10081E080936E01789480915B0184
:101C400090915C01892B09F07BC00E94F813EC0194
:101C500090935C0180935B01009709F460C06BA1D5
:101C60007CA18DA19EA160937701709378018093F0
:101C7000790190937A01EBA4FCA40DA51EA5A801FF
:101C8000970155954795379527952E0D3F1D401F78
:101C9000511F20937B0130937C0140937D01509331
:101CA0007E0120E031E742E050E020937301309361
:101CB000740140937501509376010E94EA0C8D8562
:101CC0009E85AF85B889B595A79597958795B09569
:101CD000A095909581959F4FAF4FBF4F80935E0128
:101CE00090935F01A0936001B093610180936201C2
:101CF00090936301A0936401B093650180936601A2
:101D000090936701A0936801B093690110926A01F2
:101D100010926B0110926C0110926D0111C0109223
:101D20007F0180916F008D7F80936F008AEF90E03C
:101D300020E931E0F9013197F1F70197D9F7289AB5
:101D4000E0915B01F0915C01309709F4D0C16081B2
:101D500060935D0120915E0130915F0140916001CF
:101D60005091610181819281A381B481280F391F33
:101D70004A1F5B1F20935E0130935F014093600117
:101D80005093610112161306140615069CF4646044
:101D900060935D0185859685A785B089281B390BE1
:101DA0004A0B5B0B20935E0130935F01409360010F
:101DB000509361012091620130916301409164016F
:101DC0005091650185819681A781B085280F391FC3
:101DD0004A1F5B1F209362013093630140936401AB
:101DE000509365011216130614061506ACF4809183
:101DF0005D01886080935D0185859685A785B089A2
:101E0000281B390B4A0B5B0B209362013093630153
:101E10004093640150936501209166013091670100
:101E2000409168015091690181859285A385B485AF
:101E3000280F391F4A1F5B1F2093660130936701EB
:101E40004093680150936901121613061406150693
:101E5000ACF480915D01806180935D0185859685FC
:101E6000A785B089281B390B4A0B5B0B20936601B1
:101E700030936701409368015093690120916A0192
:101E800030916B0140916C0150916D012F5F3F4F7C
:101E90004F4F5F4F20936A0130936B0140936C0169
:101EA00050936D0185859685A785B08928173907D8
:101EB0004A075B0708F015C187A590A9A1A9B2A997
:101EC000281739074A075B0708F054C020916F01B3
:101ED00030917001409171015091720180917301B4
:101EE00090917401A0917501B0917601280F391F6E
:101EF0004A1F5B1F20937301309374014093750157
:101F000050937601213082EE380784E0480780E064
:101F1000580708F4ECC02050324E44405040209303
:101F2000730130937401409375015093760183A53A
:101F300094A5A5A5B6A5209177013091780140918F
:101F4000790150917A01820F931FA41FB51F8093CE
:101F5000770190937801A0937901B0937A0127A932
:101F600030AD41AD52AD82179307A407B50708F411
:101F700091C088C083A994A9A5A9B6A92817390733
:101F80004A075B0708F48FC0281739074A075B0721
:101F900069F480E091E7A2E0B0E080937301909350
:101FA0007401A0937501B0937601A1C020916F01D7
:101FB00030917001409171015091720180917301D3
:101FC00090917401A0917501B0917601280F391F8D
:101FD0004A1F5B1F20937301309374014093750176
:101FE00050937601213082EE380784E0480780E084
:101FF000580708F47CC02050324E44405040209393
:1020000073013093740140937501509376012091D0
:102010007701309178014091790150917A01809156
:102020007B0190917C01A0917D01B0917E0182178E
:102030009307A407B50748F483A594A5A5A5B6A55D
:10204000281B390B4A0B5B0B04C0569547953795F7
:10205000279520937701309378014093790150932D
:102060007A0127A130A541A552A5809177019091D1
:102070007801A0917901B0917A0182179307A407A2
:10208000B50740F4209377013093780140937901AC
:1020900050937A0160917701709178018091790174
:1020A00090917A011BC027A930AD41AD52AD80910E
:1020B000770190917801A0917901B0917A0182170E
:1020C0009307A407B50799F020937701309378011F
:1020D0004093790150937A01CA01B9010E94EA0C38
:1020E00006C010925C0110925B010E94E91380917E
:1020F0005D019091EA06892780935D0110926E013F
:10210000FF91EF91DF91CF91BF91AF919F918F910F
:102110007F916F915F914F913F912F911F910F91FF
:10212000FF90EF900F900FBE0F901F901895F999A8
:10213000FECF92BD81BD81E08FBB80B50895F8943C
:10214000F999FECF92BD81BD81E08FBB40B5462796
:10215000842F992787FD9095262F30E082239323A3
:10216000892B39F06F3F19F060BD84E006C084E12F
:1021700004C0442321F060BD84E28FBBF99A7894B7
:1021800008958F929F92AF92BF92CF92DF92EF927B
:10219000FF920F93DF93CF9300D0CDB7DEB75C01F2
:1021A0006B017A014A0100E01EC0002319F021E012
:1021B00030E008C0202F332727FD30952227330F2A
:1021C000221F3327F60161916F01062F020F9C0138
:1021D0002F5F3F4F3A8329830E949F100894810804
:1021E000910889819A8181149104F9F6C7018A0DB9
:1021F0009B1D602F0E949F100F900F90CF91DF9139
:102200000F91FF90EF90DF90CF90BF90AF909F9095
:102210008F900895CF93DF93EC01FB019A0190E03A
:10222000B1E019C0F999FECFF2BDE1BDBFBBA0B5C9
:10223000992319F081E090E008C0892F992787FD44
:1022400090958827990F881F992731969A2F980F74
:10225000A993215030402115310521F7460F571F12
:10226000F999FECF52BD41BD81E08FBB80B520E022
:1022700030E0981711F421E030E0C901DF91CF91EF
:10228000089580E090E064E00E949F1081E090E07B
:1022900064ED76E043E250E00E94C1100895EF92B1
:1022A000FF920F931F93CF93DF93EC017A018B0181
:1022B0008530910509F455C08630910554F483307A
:1022C000910581F1843091050CF042C097FF12C056
:1022D00086C08730910509F456C0873091050CF40B
:1022E00049C08830910509F457C08930910509F03B
:1022F00076C069C0CB01BA0120E030E040E050E098
:102300000E94831E18161CF089ED91E06FC0CC0F5F
:10231000DD1FCC0FDD1FCC52D94FE882F9820A8332
:102320001B8360C0CB01BA0120E030E040E450E400
:102330000E94831E88231CF482EB91E057C0C801E1
:10234000B7010E94C6210E94F71E6093E1064AC0B1
:102350004093E2065093E3066093E4067093E5062B
:1023600041C04093E6065093E7066093E8067093F9
:10237000E90638C04093EB065093EC066093ED06F7
:102380007093EE062FC0CB01BA010E943D220E943D
:10239000F71E6093EA0626C0CB01BA0120E030E0C8
:1023A00040E752E40E94632120E030E040E752E43D
:1023B0000E9463216093EF067093F0068093F1060C
:1023C0009093F2060FC0DB01CA01BF778093F3063A
:1023D0009093F406A093F506B093F60603C08EE939
:1023E00091E004C00E94411189E891E00E949B1D88
:1023F000DF91CF911F910F91FF90EF9008951F9360
:1024000080E090E00E949710182F843081F484EDD2
:1024100096E061E070E043E250E00E940A1120E0A3
:10242000892B09F421E081E0282730E05EC081306B
:1024300021F584ED96E061E070E04BE150E00E9410
:102440000A11892B09F44FC080E098ECAFE2B8E4A0
:102450008093EF069093F006A093F106B093F206F6
:102460008DEC9CECACE4BDE38093F3069093F40612
:10247000A093F506B093F60631C08250823098F5ED
:1024800084ED96E061E070E043E250E00E940A11C2
:10249000892B49F1123061F48DEC9CECACE4BDE386
:1024A0008093F3069093F406A093F506B093F60696
:1024B0006091EF067091F0068091F1069091F2061E
:1024C00020E030E041E655E40E9463216093EF068E
:1024D0007093F0068093F1069093F2060E944111EA
:1024E00021E030E002C020E030E0C9011F910895F2
:1024F0008CE693E00E949B1D6091D4067091D506F6
:102500008091D6069091D7060E94081D87E593E03A
:102510000E949B1D6091D8067091D9068091DA06C1
:102520009091DB060E94081D82E493E00E949B1DAF
:102530006091DC067091DD068091DE069091DF06E9
:102540000E94081D8DE293E00E949B1D6091E106B0
:1025500070E080E090E00E947B1D8BE093E00E94A1
:102560009B1D6091E2067091E3068091E4069091D4
:10257000E5060E94081D88EE92E00E949B1D609176
:10258000E6067091E7068091E8069091E9060E94C0
:10259000081D85EC92E00E949B1D6091EB067091F6
:1025A000EC068091ED069091EE060E94081D8CEAE3
:1025B00092E00E949B1D6091EA0670E080E090E04E
:1025C0000E947B1D89E892E00E949B1D6091EA06B3
:1025D00070E080E090E022E030E040E050E00E94D7
:1025E000811C80E892E00E949B1D6091EF06709133
:1025F000F0068091F1069091F20620E030E041E68D
:1026000055E40E948A1E0E94081D8DE592E00E94FA
:102610009B1D6091F3067091F4068091F5069091F0
:10262000F6060E94081D87E392E00E949B1D82EF40
:1026300091E00E949B1D08950E94FF11892B29F0B3
:102640008AE691E00E949B1D08958FE291E00E942E
:102650009B1D84EF99EFACE3B4E48093D406909390
:10266000D506A093D606B093D7068093D80690934C
:10267000D906A093DA06B093DB068093DC0690932C
:10268000DD06A093DE06B093DF068EE18093E106BF
:1026900080E090E0AAEFB3E48093E2069093E30633
:1026A000A093E406B093E5068093E6069093E706D0
:1026B000A093E806B093E90680E098ECAFE2B8E4B6
:1026C0008093EF069093F006A093F106B093F20684
:1026D0008DEC9CECACECBDE38093EB069093EC06A8
:1026E000A093ED06B093EE068CE18093EA068DECA4
:1026F0009CECACE4BDE38093F3069093F406A093C6
:10270000F506B093F6060E9441110E9478120895D2
:10271000EF92FF920F931F93DF93CF93CDB7DEB766
:1027200029970FB6F894DEBF0FBECDBF8C0181E0B4
:102730008983F80180818432E1F58181882319F44D
:102740000E94781234C0C8017E010894E11CF11C7B
:10275000B701AE014E5F5F4F0E94991B892B59F163
:102760009981F801E90FF11D80818D3311F59F5F8B
:102770009983C801B701AE014A5F5F4F0E94991B60
:10278000892BC9F08981080F111DF80180818823E8
:1027900081F46A817B818C819D810E94F21EDC0123
:1027A000CB014E815F81688579850E944F1180E061
:1027B00003C083E001C081E029960FB6F894DEBF24
:1027C0000FBECDBFCF91DF911F910F91FF90EF9082
:1027D00008959091A6058091A705981741F08091E2
:1027E000A7058F5F823109F480E08093A7050895E3
:1027F0009091A6058091A705981719F420E030E084
:1028000008C09091A7058BE3989F90011124205850
:102810003E4FC90108958F929F92AF92BF92CF927F
:10282000DF92EF92FF920F931F9349015A0120917B
:10283000D4063091D5064091D6065091D7060E9415
:1028400063210E94332128EAC22E25E0D22E609314
:10285000A8057093A9058093AA059093AB05C501BF
:10286000B4012091D8063091D9064091DA065091F2
:10287000DB060E9463210E943321F60134966093A7
:10288000AC05718382839383C801B7012091DC0674
:102890003091DD064091DE065091DF060E946321F3
:1028A0000E94332128E030E0C20ED31E6093B005B1
:1028B000D60111967C93119712968C9312971396CA
:1028C0009C9380E090E0A0E0B0E08093C0059093FE
:1028D000C105A093C205B093C3058CE0E4EBF5E01D
:1028E000DF011D928A95E9F71F910F91FF90EF90FC
:1028F000DF90CF90BF90AF909F908F9008951092EF
:10290000A6051092A7058CE0E8EAF5E0DF01982F14
:102910001D929A95E9F7E4EBF5E0DF011D928A95A7
:10292000E9F780E090E0A0E0B0E08093C0059093EC
:10293000C105A093C205B093C30508958F929F92DD
:10294000AF92BF92CF92DF92EF92FF920F931F93BD
:10295000CF93DF93EC016B01009709F460C08AA16B
:10296000882309F05CC0ED88FE880F89188DFB0173
:10297000B588A6889788808CC801B7012B2D3A2D81
:10298000492D582D0E94831E88230CF048C0C80191
:10299000B701A80197010E9463217B018C0160911E
:1029A000EF067091F0068091F1069091F206905832
:1029B00020E030E040E050EC0E9463212D8D3E8D00
:1029C0004F8D58A10E9463219B01AC01C801B70142
:1029D0000E94AA1D0E94F0217B018C016B2D7A2D93
:1029E000892D982D9701A8010E94831E882324F425
:1029F000EB2CFA2C092D182D6B2D7A2D892D982D65
:102A00009701A8010E94831E882349F0C701D801BD
:102A1000F601858B968BA78BB08F81E081A3DF9128
:102A2000CF911F910F91FF90EF90DF90CF90BF90CB
:102A3000AF909F908F9008952F923F924F925F9208
:102A40006F927F928F929F92AF92BF92CF92DF92BE
:102A5000EF92FF920F931F93DF93CF93CDB7DEB723
:102A600068970FB6F894DEBF0FBECDBF1C016A0198
:102A70007B0128013901DC01D7966D917D918D9103
:102A80009C91DA970E94231F4B015C01A7019601DC
:102A90000E9463210E94701E0E94F71E7B018C0120
:102AA000F10163A374A385A396A3C501B401A30197
:102AB00092010E9463210E94701E0E94F71E698786
:102AC0007A878B879C87D10197966D937D938D93A1
:102AD0009C939A979B966D917D918D919C919E97D9
:102AE00022E330E040E050E00E9460220E94251F77
:102AF00020E030E040E752E40E9463210E94F21E91
:102B00002B013C01C801B7010E94231F7B018C01EE
:102B1000C301B2010E94251F6D837E838F83988736
:102B2000C501B401A50194010E9463215B016C0100
:102B3000C801B701A80197010E9463216D877E87B4
:102B40008F87988B6D817E818F8198859B01AC01E9
:102B50000E94AA1D698B7A8B8B8B9C8BC601B50159
:102B60002D853E854F8558890E94A91D29893A895E
:102B70004B895C890E948A1E0E94701E0E94F21E70
:102B800069837A838B839C8369857A858B859C8511
:102B90000E94231F9B01AC010E9463216D8B7E8BE1
:102BA0008F8B988FA60195010E94A91D7B018C0136
:102BB0007094609450944094411C511C611C711C91
:102BC000C301B2010E94251F9B01AC010E94AA1DF6
:102BD0009B01AC01C801B7010E948A1E0E94601FC0
:102BE000F101A584B684C784D08886017501298146
:102BF0003A814B815C81E21AF30A040B150B0E94A7
:102C0000F21EA8019701261B370B480B590BDA015E
:102C1000C90157FF4AC0C601B5010E94251F9B018B
:102C2000AC0169897A898B899C890E9463212D85F1
:102C30003E854F8558890E94A91D2D893E894F895F
:102C4000588D0E94AA1D7B018C016D817E818F8130
:102C5000988520E030E040E850E40E9463219B0129
:102C6000AC01C801B7010E948A1E0E94701E0E941A
:102C7000F21EAC01CB01DA01BC01CD0197FF04C00B
:102C800060E070E080E090E069837A838B839C83CE
:102C9000A616B706C806D90624F4A982BA82CB8242
:102CA000DC8280E090E0A0E0B0E029813A814B81B5
:102CB0005C81F10127A730AB41AB52AB820F931F70
:102CC000A41FB51F83AB94ABA5ABB6AB68960FB68C
:102CD000F894DEBF0FBECDBFCF91DF911F910F9152
:102CE000FF90EF90DF90CF90BF90AF909F908F902C
:102CF0007F906F905F904F903F902F9008952F920C
:102D00003F924F925F926F927F928F929F92AF927B
:102D1000BF92CF92DF92EF92FF920F931F93DF93B8
:102D2000CF93CDB7DEB7CC54D0400FB6F894DEBF0A
:102D30000FBECDBF29013A01ACAEBDAECEAEDFAE07
:102D400021968FAE21972091D4063091D5064091DF
:102D5000D6065091D70628AF39AF4AAF5BAF0E9475
:102D600063210E94332122966FAF229723967FAF73
:102D7000239724968FAF249725969FAF2597809110
:102D8000D8069091D906A091DA06B091DB068CABFB
:102D90009DABAEABBFABC301B2012CA93DA94EA9FF
:102DA0005FA90E9463210E94332126966FAF269768
:102DB00027967FAF279728968FAF289729969FAFA2
:102DC00029972091DC063091DD064091DE06509176
:102DD000DF0628AB39AB4AAB5BABC801B7010E9439
:102DE00063210E9433212A966FAF2A972B967FAFDB
:102DF0002B972C968FAF2C972D969FAF2D973091B8
:102E0000A6053F5F3B8F323149F41B8E07C083B765
:102E1000816083BF889583B78E7F83BF8091A7052C
:102E20004B8D8417A1F39091A6058BE3989FD00159
:102E30001124A058BE4FBA8FA98F1C922091A805CB
:102E40003091A9054091AA055091AB0525968CAD0E
:102E50009DADAEADBFAD259782179307A407B5070B
:102E600024F480E2A98DBA8D8C936090AC057090AB
:102E7000AD058090AE059090AF0529968CAD9DADC7
:102E8000AEADBFAD299786159705A805B9052CF4F9
:102E9000A98DBA8D8C9180648C93E090B005F090F0
:102EA000B1050091B2051091B3052D968CAD9DAD85
:102EB000AEADBFAD2D978E159F05A007B1072CF4C1
:102EC000A98DBA8D8C9180688C932596ACACBDACE5
:102ED000CEACDFAC2597A21AB30AC40AD50AE98D95
:102EE000FA8DA182B282C382D482D7FE0BC088271A
:102EF0009927DC018A199B09AC09BD09818392835A
:102F0000A383B48329962CAD3DAD4EAD5FAD29971B
:102F1000261937094809590939014A01A98DBA8D7D
:102F200015962D933D934D935C93189757FF0DC0C5
:102F300088279927DC01821B930BA40BB50BE98D25
:102F4000FA8D85839683A783B0872D962CAC3DACF4
:102F50004EAC5FAC2D972E183F08400A510AA201D3
:102F6000910157FE07C022273327A90122193309EF
:102F700044095509A98DBA8D19962D933D934D930A
:102F80005C931C971596ED90FD900D911C911897F0
:102F9000FD0181819281A381B4818E159F05A007D7
:102FA000B10710F4D801C70182179307A407B5072A
:102FB00010F4DA01C901E98DFA8D85879687A78714
:102FC000B08B0097A105B10509F486C3C601B50110
:102FD0000E94251F28AD39AD4AAD5BAD0E948A1E07
:102FE0006CA77DA78EA79FA7C401B3010E94251FD0
:102FF0002CA93DA94EA95FA90E948A1E68A779A79E
:103000008AA79BA7C201B1010E94251F28A939A93F
:103010004AA95BA90E948A1E6CA37DA38EA39FA3CD
:103020006CA57DA58EA59FA50E943A223B014C016F
:1030300068A579A58AA59BA50E943A227B018C01EF
:103040006CA17DA18EA19FA10E943A225B016C011F
:10305000C401B301A80197010E94AA1DA601950110
:103060000E94AA1D0E94F0217B018C01A98DBA8DBE
:103070005D966D937D938D939C93909760E070E047
:1030800080E89FE3A80197010E948A1E3B014C0142
:103090002196BFAD2197BB2349F46CAD7DAD8EADBC
:1030A0009FADA40193010E9463210AC060E070E01B
:1030B00080E89FE32CAD3DAD4EAD5FAD0E948A1E12
:1030C0005B016C01C801B701A60195010E94632153
:1030D0001B012C01E98DFA8D618B728B838B948B94
:1030E00065857685878590890E94251F7B018C01E7
:1030F000A60195010E9463210E94701E0E94F71E86
:10310000A98DBA8DD7966D937D938D939C93DA9705
:103110002091EF063091F0064091F1065091F206B1
:1031200028A339A34AA35BA3C801B701A401930153
:103130000E94632128A139A14AA15BA10E946321B9
:1031400020E030E84BE355E40E948A1E0E94701E86
:103150000E94F21EA98DBA8D9B966D937D938D93DF
:103160009C939E976CA57DA58EA59FA5A401930118
:103170000E9463217B018C016D877E878F87988BEE
:1031800068A579A58AA59BA5A40193010E94632146
:103190005B016C01698B7A8B8B8B9C8B6CA17DA105
:1031A0008EA19FA1A40193010E9463216C8F7D8F4A
:1031B0008E8F9F8F9091A6058091A705981709F48F
:1031C000ADC06090C0057090C1058090C205909020
:1031D000C305B301C40120E030E040E050E00E94AC
:1031E000912018160CF09AC06091B4057091B50545
:1031F0008091B6059091B7059058A80197010E945B
:1032000063217B018C01C601B5012091B805309185
:10321000B9054091BA055091BB050E9463219B01FD
:10322000AC01C801B7010E94A91D7B018C016C8D06
:103230007D8D8E8D9F8D2091BC053091BD05409177
:10324000BE055091BF050E9463219B01AC01C801DE
:10325000B7010E94A91D7B018C0123E333E343E7FF
:103260005FE30E94831E88230CF058C0B301C401A1
:10327000A20191010E94831E87FD04C0D201C101F9
:1032800031014D01C801B70123E333E343E75FEBAD
:103290000E94912018160CF046C060E070E080E8B3
:1032A0009FE3A80197010E94A91D20E030E040E0C3
:1032B0005FE30E9463210E94F0215B016C0168A121
:1032C00079A18AA19BA12091F3063091F406409147
:1032D000F5065091F6060E946321A60195010E9411
:1032E00063217B018C0160E070E080E89FE3A60130
:1032F00095010E94A91D9B01AC01C801B7010E9464
:103300008A1E0E94F0217B018C01B301C401970148
:10331000A8010E94831E87FD06C007C0EE24FF247B
:1033200000E010E002C073018401C701D801E98DFB
:10333000FA8D818F928FA38FB48F68A179A18AA112
:103340009BA1905820E030E040E050EC0E946321C7
:10335000A98DBA8D5D962D913D914D915C9190977F
:103360000E94632120E030E040E050E00E94AA1D6E
:103370000E94F021D62EC72EB82EA92EB701C80163
:103380002D2D3C2D4B2D5A2D0E94831E87FD04C0F0
:10339000ED2CFC2C0B2D1A2DC701D801E98DFA8DCF
:1033A000858B968BA78BB08F61897289838994896D
:1033B0002D2D3C2D4B2D5A2D0E94831E181634F0B6
:1033C00081E0A98DBA8D92968C9303C0E98DFA8D18
:1033D00012A281E0A98DBA8D91968C932C8D3D8D92
:1033E0004E8D5F8D2D8B3E8B4F8B588F2D968CADD8
:1033F0009DADAEADBFAD2D9789879A87AB87BC8752
:1034000029962CAD3DAD4EAD5FAD29972D833E8302
:103410004F83588725968CAD9DADAEADBFAD25973A
:1034200089839A83AB83BC83A4EBB5E0FE013D9610
:103430008CE001900D928150E1F7E98DFA8D818940
:103440009289A389B4898093C0059093C105A09304
:10345000C205B093C305FB8DF093A605A8EAB5E0BD
:10346000FE0131968CE001900D928150E1F7709051
:10347000A6058091EF069091F006A091F106B0911B
:10348000F2061C012D0157FA509457F85094CC24A1
:10349000DD2400E010E07BE3672E87C0772011F485
:1034A00062E1762E7A94C114D10409F474C0011536
:1034B000110509F470C0D6015996BC9059975A96D7
:1034C000AC905A975B969C905B975C968C905C97BF
:1034D00055966D917D918D919C9158972B2D3A2DFC
:1034E000492D582D0E94831E882309F454C0F601EB
:1034F00082A1882309F042C0D8015596ED90FD9035
:103500000D911C9158976B2D7A2D892D982DA8011E
:1035100097010E94912018168CF5C801B701A801E7
:1035200097010E9463217B018C01C201B10120E05F
:1035300030E040E050EC0E946321F601258D368D8D
:10354000478D50A10E9463219B01AC01C801B701C6
:103550000E94AA1D0E94F021162F072FF82EE92E97
:103560006B2D7A2D892D982D212F302F4F2D5E2DEB
:103570000E94831E87FD02C0580147018B2D9A2DA2
:10358000A92DB82DF601858B968BA78BB08FE1E026
:10359000D6019196EC93769CC0011124860150E8E7
:1035A000C52E51E0D52EC80ED91E8091A7057816DC
:1035B00009F074CFD090A705EE24FF2420E030E07E
:1035C0004BE3C42E11C0DC9C8001112400581E4F17
:1035D000C901B701A8010E949E14D394F2E1DF163D
:1035E00009F4DD24970178018091A605D81659F7D2
:1035F000C901B70140E050E00E949E145090A70519
:10360000882499243BE3432E3FC0549C300111246D
:1036100020E831E0620E731E8114910479F1D40127
:1036200091968C91882321F4F30181A1882331F1B3
:10363000D4015196ED90FD900D911C9154975596A3
:103640006D917D918D919C915897A80197010E9451
:103650008A1E5B016C01F301658976898789908DEB
:10366000A80197010E948A1E8B019C01C401B6012A
:10367000A5010E941C15D40191961C925394B2E1AD
:103680005B1609F4552443018091A605581609F0EC
:10369000BCCFF401E188F2880389148965897689B1
:1036A0008789908DA80197010E948A1E5B016C0199
:1036B00060E070E080E090E0A80197010E948A1E1F
:1036C0008B019C01C401B601A5010E941C15D40107
:1036D00091961C920E94AC0DC45BDF4F0FB6F8941C
:1036E000DEBF0FBECDBFCF91DF911F910F91FF9035
:1036F000EF90DF90CF90BF90AF909F908F907F9092
:103700006F905F904F903F902F90089520EA3FE098
:1037100004C0F9013197F1F701970097D1F70895A7
:1037200035E004C0232F2A95F1F701970097D1F7D0
:103730000895AF92BF92CF92DF92EF92FF920F93D4
:103740001F93DF93CF9300D0CDB7DEB76C015B0141
:103750007A01FB0180818601080F111DC801BE019D
:103760006F5F7F4F0E94F601F70160837183828350
:10377000938389819A818017910719F420E030E0C2
:1037800005C08C19F501808321E030E0C9010F905C
:103790000F90CF91DF911F910F91FF90EF90DF90ED
:1037A000CF90BF90AF90089584B1817F84B9089580
:1037B0006F927F928F929F92AF92BF92CF92DF9241
:1037C000EF92FF920F931F93982EA62EB42E6701AF
:1037D00078018091E106C81AD108E108F108992022
:1037E00011F094EE01C090EEA1109860B1109061BC
:1037F000222311F080EE98270091EA0609278BB169
:10380000902F907E8F71982B9BB924E0622E98E0C8
:10381000792E80E1882E83B1992021F0199902C078
:1038200006259924AA2021F01A9902C00725AA2466
:10383000BB2021F01B9902C00825BB24992021F44C
:10384000AA2011F4BB2089F08BB1102F1C71812BA1
:103850008BB98091E10690E00E94901B8BB11827F4
:103860001BB9C6010E94901BD6CF1F910F91FF90EC
:10387000EF90DF90CF90BF90AF909F908F907F9010
:103880006F900895DF92EF92FF920F931F930E9423
:10389000D30DD3B080E060E041E020E0F0EAEF2E0D
:1038A000F6E8FF2EF1E00F2F112D0E94D81B81E0CA
:1038B00061E040E020E00E94D81B83B18D258E702E
:1038C00090E0BC0176956795769567956170AC013F
:1038D00073E0569547957A95E1F7417096958795EF
:1038E000817021E030E2E32E31EAF32E37E0032F3E
:1038F000112D0E94D81B1F910F91FF90EF90DF9028
:1039000008952F923F924F925F926F927F928F9283
:103910009F92AF92BF92CF92DF92EF92FF920F935E
:103920001F93DF93CF93CDB7DEB7A0970FB6F89470
:10393000DEBF0FBECDBF6B017C0129013A016115CD
:1039400071058105910521F480E30E94C40B47C0F5
:103950008824992454011E010894211C311C8101E2
:10396000080D191DC701B601A30192010E947F2213
:10397000F80160830894811C911CA11CB11CC70133
:10398000B601A30192010E947F22C901DA016C01F4
:103990007D01C114D104E104F10409F77101E80CBF
:1039A000F91C3E010894611C711CD501C4010197EA
:1039B000A109B1096C01C818D9080EC0F601EE0DB5
:1039C000FF1D80818A3010F4805D01C0895C0E94F7
:1039D000C40B0894E108F1086E147F0479F7A096EF
:1039E0000FB6F894DEBF0FBECDBFCF91DF911F9110
:1039F0000F91FF90EF90DF90CF90BF90AF909F908E
:103A00008F907F906F905F904F903F902F90089590
:103A1000AF92BF92CF92DF92EF92FF920F931F93DC
:103A2000CF93DF937B018C0120E030E040E050E059
:103A30000E94831E88233CF48DE20E94C40B17FB76
:103A4000109517F91095C801B7012FE632E143E050
:103A50005AE30E94AA1D7B018C010E94F21E5B01A9
:103A60006C01CC24B7FCC094DC2CC601B5012AE063
:103A700030E040E050E00E94811C8EE20E94C40BC6
:103A8000C601B5010E94251F9B01AC01C801B70109
:103A90000E94A91DC3E0D0E01EC020E030E040E25B
:103AA00051E40E9463215B016C010E94F21E7B01C4
:103AB0008C01862F805D0E94C40B6E2D70E08827DC
:103AC00077FD8095982F0E94251F9B01AC01C601B0
:103AD000B5010E94A91D21972FEFCF3FD207E9F62C
:103AE000DF91CF911F910F91FF90EF90DF90CF90DA
:103AF000BF90AF900895EF92FF920F931F937B01B9
:103B00008C0197FF0BC08DE20E94C40B10950095AD
:103B1000F094E094E11CF11C011D111DC801B701D6
:103B20002AE030E040E050E00E94811C1F910F919C
:103B3000FF90EF900895CF93DF93EC0102C00E94B5
:103B4000C40BFE01219684918823C9F7DF91CF91A0
:103B500008955058BB27AA270ED081C241D230F019
:103B600046D220F031F49F3F11F41EF411C20EF43E
:103B7000E095E7FBDCC1E92F94D280F3BA17620726
:103B800073078407950718F071F49EF5C3C20EF40D
:103B9000E0950B2EBA2FA02D0B01B90190010C015D
:103BA000CA01A0011124FF27591B99F0593F50F475
:103BB000503E68F11A16F040A22F232F342F4427CD
:103BC000585FF3CF469537952795A795F0405395C5
:103BD000C9F77EF41F16BA0B620B730B840BBAF095
:103BE0009150A1F0FF0FBB1F661F771F881FC2F700
:103BF0000EC0BA0F621F731F841F48F48795779514
:103C00006795B795F7959E3F08F0B3CF9395880FCA
:103C100008F09927EE0F979587950895E1D158F010
:103C200080E891E009F49EEFE2D128F040E851E00D
:103C300059F45EEF09C0ACC16DC2E92FE07831D212
:103C400068F3092E052AC1F32617370748075907D5
:103C500038F00E2E07F8E02569F0E025E0640AC090
:103C6000EF6307F8009407FADB01B9019D01DC015D
:103C7000CA01AD01EF935DD0F2D10AD05F91552317
:103C800031F02BED3FE049E450FD49EC63CF08955E
:103C9000DF93DD27B92FBF7740E85FE316161706DD
:103CA00048075B0710F4D92FA1D29F938F937F937E
:103CB0006F93E0D3E8E6F0E06ED1D1D12F913F9140
:103CC0004F915F910CD3DD2349F09058A2EA2AED81
:103CD0003FE049EC5FE3D0785D274DDFDF91BFC166
:103CE00002D280F09F3740F491110EF414C260E0CC
:103CF00070E080E89FE3089526F01B16611D711D9A
:103D0000811D1BC135C1EFD008F481E0089577D142
:103D1000E395B6C10CD0A3C16AD140F061D130F0B7
:103D200021F45F3F19F003C15111F5C131C1B9D17F
:103D300098F39923C9F35523B1F3951B550BBB2772
:103D4000AA2762177307840738F09F5F5F4F220F1F
:103D5000331F441FAA1FA9F333D00E2E3AF0E0E818
:103D600030D091505040E695001CCAF729D0FE2F64
:103D700027D0660F771F881FBB1F261737074807F6
:103D8000AB07B0E809F0BB0B802DBF01FF279358AC
:103D90005F4F2AF09E3F510568F0C9C0BCC15F3F2C
:103DA000ECF3983EDCF3869577956795B795F79594
:103DB0009F5FC9F7880F911D9695879597F908958C
:103DC000E1E0660F771F881FBB1F62177307840728
:103DD000BA0720F0621B730B840BBA0BEE1F88F737
:103DE000E095089504D06894B11195C1089561D10A
:103DF00088F09F5790F0B92F9927B751A0F0D1F0D4
:103E0000660F771F881F991F1AF0BA95C9F712C05D
:103E1000B13081F07FD1B1E008957CC1672F782F58
:103E20008827B85F39F0B93FCCF3869577956795C9
:103E3000B395D9F73EF490958095709561957F4F35
:103E40008F4F9F4F0895E89409C097FB3EF49095DB
:103E50008095709561957F4F8F4F9F4F9923A9F063
:103E6000F92F96E9BB279395F695879577956795F2
:103E7000B795F111F8CFFAF4BB0F11F460FF1BC036
:103E80006F5F7F4F8F4F9F4F16C0882311F096E9C9
:103E900011C0772321F09EE8872F762F05C0662377
:103EA00071F096E8862F70E060E02AF09A95660F30
:103EB000771F881FDAF7880F9695879597F90895E9
:103EC00012D180F09F3740F491110EF024C160E0D0
:103ED00070E080E89FEB089526F41B16611D711DAC
:103EE000811D2BC045C0990F0008550FAA0BE0E8B3
:103EF000FEEF16161706E807F907C0F012161306AC
:103F0000E407F50798F0621B730B840B950B39F4EB
:103F10000A2661F0232B242B252B21F408950A2651
:103F200009F4A140A6958FEF811D811D089597F991
:103F30009F6780E870E060E00895882371F477233C
:103F400021F09850872B762F07C0662311F499270C
:103F50000DC09051862B70E060E02AF09A95660FB4
:103F6000771F881FDAF7880F9695879597F9089538
:103F70009F3F49F0915028F4869577956795B795BE
:103F80009F5F80389F4F880F9695879597F9089582
:103F90009FEF80EC0895DF93CF931F930F93FF92D1
:103FA000EF92DF927B018C01689405C0DA2EEF015D
:103FB00096D1FE01E894A5912591359145915591B1
:103FC000AEF3EF01D8DDFE019701A801DA9479F78D
:103FD000DF90EF90FF900F911F91CF91DF910895A7
:103FE00000240A94161617061806090608950024D8
:103FF0000A9412161306140605060895C9CF59D05F
:10400000E8F3E894EFEFBB273FE048EC5FE76B3D58
:1040100073078407950708F1FF279F57B25A6A4D27
:104020007F40894CF04032F4BE556542704F864364
:10403000FF4F0894EE1F915030F0BB0F661F771FA3
:10404000881FFF1FEBCF9EE7882332F0BB0F661F50
:10405000771F881F9A95C1F79395E09589CF092E10
:104060000394000C11F4882352F0BB0F40F4BF2BD3
:1040700011F460FF04C06F5F7F4F8F4F9F4F089513
:10408000EF93E0FF06C0A2EA2AED3FE049EC5FEBC8
:1040900072DDE5DF0F90039401FC9058E5E9F0E054
:1040A000FEC157FD9058440F551F59F05F3F71F006
:1040B0004795880F97FB991F61F09F3F79F087958F
:1040C0000895121613061406551FF2CF4695F1DF18
:1040D00008C0161617061806991FF1CF86957105A8
:1040E000610508940895E5DFA0F0BEE7B91788F4EC
:1040F000BB279F3860F41616B11D672F782F8827CD
:10410000985FF7CF869577956795B11D939596390A
:10411000C8F30895E894BB2766277727CB0197F962
:104120000895E1DE08F48FEF08955ADF19F05FDF9C
:1041300009F02ECFFCCEB901CA011ACF9F775F7765
:10414000B0DF98F39923B9F35523B9F3FF279517F7
:1041500058F4E52FE91BED3070F75E3B10F0F1E409
:104160001CC09034E0F40AC0E92FE51BED3028F7BD
:104170009E3B10F0F1E411C0503488F4F9EA882332
:104180002AF09A95660F771F881FDAF744232AF0E2
:104190005A95220F331F441FDAF79F1B5F1BFF93B3
:1041A0001F930F93FF92EF9279018A01BB27AB2FE8
:1041B0009B01AC0196D09701A801BF937B018C01B4
:1041C000AA27BA2FB901CA018CD0AF919701A801D3
:1041D000EF90FF900F911F91CEDC41DF01D14F9105
:1041E00040FF0895552747FD509509C09B01AC013C
:1041F00060E070E080E89FE38DCD99CEB9CE59DFC5
:10420000E8F39923D9F3940F511DBBF3915050401B
:1042100094F059F0882332F0660F771F881F915071
:104220005040C1F79E3F510544F7880F911D969568
:10423000879597F908955F3FACF0983E9CF0BB27B7
:10424000869577956795B79508F4B1609395C1F712
:10425000BB0F58F711F460FFE8CF6F5F7F4F8F4FB0
:104260009F4FE3CF58CF25DF58F19E5758F1985113
:10427000A0F0E9F0983020F5092E9927660F771FF6
:10428000881F991F0A94D1F712C0062E672F782F26
:104290008827985F11F4000C07C0993FB4F3869506
:1042A000779567959395D9F7611D711D811D3EF432
:1042B00090958095709561957F4F8F4F9F4F089592
:1042C000689429CF27CF0BD0CACE8ADE28F08FDEA4
:1042D00018F0952309F02BCE5BCE11241CCFE1DE24
:1042E000A0F3959FD1F3950F50E0551F629FF00109
:1042F000729FBB27F00DB11D639FAA27F00DB11D62
:10430000AA1F649F6627B00DA11D661F829F2227EA
:10431000B00DA11D621F739FB00DA11D621F839F71
:10432000A00D611D221F749F3327A00D611D231F47
:10433000849F600D211D822F762F6A2F11249F5795
:1043400050408AF0E1F088234AF0EE0FFF1FBB1FB8
:10435000661F771F881F91505040A9F79E3F510557
:1043600070F0E5CDD8CE5F3FECF3983EDCF3869558
:1043700077956795B795F795E7959F5FC1F7FE2B02
:10438000880F911D9695879597F9089592DEE0F034
:104390009E37D8F09639B8F49E3848F4672F782FB6
:1043A0008827985FF9CF8695779567959395953986
:1043B000D0F3B62FB1706B0F711D811D20F487955E
:1043C000779567959395B9CDD3CDA5CE9F9317DEFD
:1043D0000F9007FCEE5F54CE11F40EF4D9CDC8CD8A
:1043E00068DED0F39923D9F3CEF39F57550B87FF9F
:1043F0004FD056959795B0E020F4660F771F881F31
:10440000BB1F1F930F9300249001A0018001F001B6
:10441000A0E80E0F1F1F0A1E511D601B710B8009A3
:10442000B50B48F4600F711F801DB51F0E1B1F0BCD
:104430000A0A510907C02E0F3F1F4A1F0E0F1F1FE8
:104440000A1E511D660F771F881FBB1FA695F79583
:10445000E795F8F60617170708065B07211D311DBB
:10446000411D0F911F91B901842F9158880F969586
:10447000879508959B01AC0126CF35DE20F09F374C
:1044800008F449CE5ACD74CD2EDD880B990B0895D2
:1044900091505040660F771F881FD2F708959F9361
:1044A0008F937F936F93FF93EF939B01AC010BDF8F
:1044B000EF91FF9170DD2F913F914F915F9103CF6D
:1044C000629FD001739FF001829FE00DF11D649FF8
:1044D000E00DF11D929FF00D839FF00D749FF00D84
:1044E000659FF00D9927729FB00DE11DF91F639F25
:1044F000B00DE11DF91FBD01CF0111240895A1E206
:104500001A2EAA1BBB1BFD010DC0AA1FBB1FEE1F4D
:10451000FF1FA217B307E407F50720F0A21BB30B98
:10452000E40BF50B661F771F881F991F1A9469F714
:1045300060957095809590959B01AC01BD01CF0170
:10454000089597FB092E05260ED057FD04D0D7DF1E
:104550000AD0001C38F450954095309521953F4F76
:104560004F4F5F4F0895F6F7909580957095619540
:104570007F4F8F4F9F4F0895911106C0803219F0E1
:1045800089508550D0F708959927882708952F924C
:104590003F924F925F926F927F928F929F92AF92D3
:1045A000BF92CF92DF92EF92FF920F931F93CF9320
:1045B000DF93CDB7DEB7CA1BDB0B0FB6F894DEBFB7
:1045C0000FBECDBF09942A88398848885F846E84DD
:1045D0007D848C849B84AA84B984C884DF80EE8027
:1045E000FD800C811B81AA81B981CE0FD11D0FB630
:1045F000F894DEBF0FBECDBFED010895F894FFCF54
:00000001FF
